:020000040000FA
:04000000B1EF0FF05D
:08000800056ED8CF06F0E0CF31
:1000100007F00001E9CF0DF0EACF08F0E1CF09F0D9
:10002000E2CF0AF0D9CF0BF0DACF0CF0F3CF14F017
:10003000F4CF15F0FACF16F000C00FF001C010F0A9
:1000400002C011F003C012F004C013F0F2AA2CEFAA
:1000500000F0F2B42FEF01F0A0AA32EF00F0A1BA45
:100060003AEF09F00FC000F010C001F011C002F02B
:1000700012C003F013C004F00DC0E9FF08C0EAFF8E
:10008000088E09C0E1FF0AC0E2FF0BC0D9FF0CC017
:10009000DAFF14C0F3FF15C0F4FF16C0FAFF0550D5
:1000A00007C0E0FF06C0D8FF1000F76ABA0FF66E6F
:1000B000000EF7220900F5501200000302FFFFFFB7
:1000C000FFFFFFFFFFFFFFFFFFFFF76ADA0FF66E8C
:1000D000000EF7220900F550120000FF02FFFFFF9B
:1000E000FFFFFFFFFFFFFFFFFFFFF76AFA0FF66E4C
:1000F000000EF7220900F5501200400008004000F1
:1001000000000000000000000000000000000000EF
:1001100000000000000000000000F76A2A0FF66EE1
:10012000010EF7220900F5501200400000004000C7
:1001300000000000000000000000000000000000BF
:1001400000000000000000000000F76A5A0FF66E81
:10015000010EF7220900F5501200090243000201C6
:100160000080320904000001020201000524001091
:1001700001042402020524060001052401000107F0
:100180000581030800FA09040100020A00000007C3
:100190000502024100010705820241000100F76AE1
:1001A000AE0FF66E010EF7220900F55012000200A4
:1001B000F76AC00FF66E010EF7220900F550120023
:1001C00012171B20FFFFFFFFF76AD80FF66E010E14
:1001D000F7220900F5501200120110010200004040
:1001E00061043300000101020001F76AFA0FF66EA4
:1001F000010EF7220900F550120004030904080358
:1002000043004300530018035300450052004900C7
:1002100041004C002000440045004D004F00F2CF4B
:100220000EF0F29EF76A380FF66E020EF722090002
:10023000F5500EBEF28E120074696D655B735D2021
:10024000205820205865727220205920205965724C
:100250007220205A20205A657272200A0D00010E69
:100260001926D8B01A2AD8B41B2AD8B41C2AF2945A
:1002700032EF00F06D92699468A402D06894FCD7C4
:1002800045EF09F0400E0401016F040E036F180ED4
:10029000026F880E006F046B040E076F580E066F16
:1002A0000001000C70A002D0EDDF7090689A4EEF54
:1002B00009F06A6A689254EF09F0070148514A034D
:1002C000F3CF01F0F4CF00F04B03F3500026495177
:1002D0004A03F3500020026E0001000C036A07017C
:1002E0000651700FE96E0F0E0320EA6EEF6A496B3C
:1002F00006C748F74B6B080E4A6F0001DEDF0701A7
:1003000001C0E9FF040E0224EA6EEF6A496B06C7DA
:1003100048F74B6B080E4A6F0001CFDF02C008F7A9
:1003200001C007F7040E07010727000E082307C7BF
:10033000E9FF040E0825EA6EEF6A0001000C010EC9
:100340000701056F05510F0807E305C706F7000110
:10035000C5DF0701052BF6D70001000C2E6A2D6AB8
:10036000250E2C6E800E2B6E2F6A306A080E316EB1
:10037000816B8091336A326A7C6B7D91000C07013E
:10038000196B195101080AE3036A1951290FE96E23
:10039000000E0320EA6EEF6A192BF3D70001DEDFAF
:1003A0001E6A010E1F6E1D6A000C689600D000D0F8
:1003B00000D0000C6A6A686A9F0E6B6E3D0E696E13
:1003C0006E6ABDDFDCDF160E706E68A602D0EDDF50
:1003D000FCD76D9857DF030E246E5AEF09F069843D
:1003E00068986D8260EF09F0689C66EF09F000C7BD
:1003F00025F0000CFF0E256E000C0601FE6B285246
:1004000042E0FE513F083FE32050000105E0020AB0
:1004100010E0010A1BE027D0036A2750F2CF00F753
:10042000F29E93DE070100BFF28EE8CFFFF60001D7
:100430001AD0036A2750F2CF00F7F29ED6DE0701EA
:1004400000BFF28EE8CFFFF600010DD0036A2750FF
:10045000F2CF00F7F29EB8DE070100BFF28EE8CFC0
:10046000FFF6000100D0272A28060601FE51FE2BC8
:10047000580F036AD8B0032AE96E040E0324EA6E0B
:10048000FFC6EFFFBCD7285204E1FE51400801E04F
:100490001D6AFEC600F70001AADF000C276A206A69
:1004A00004011B51010A000107E0030A0AE0010AE6
:1004B0000BE0220A22E042D0120E286E030E206EBC
:1004C0003FD0430E286E3CD0020E206E036A04011A
:1004D0001A51210FE96E000E0320EA6EEFCF27F0CC
:1004E000036A2750F2CFFDF6F29E00017EDE060180
:1004F000FDBFF28E286E000123D0036A04011A5159
:10050000F2CFFDF6F29E000153DE0601FDBFF28E32
:10051000276E273C01D00FD0036A2750F2CFFDF69B
:10052000F29E000112DE0601FDBFF28E286E000170
:1005300007D004D0060100015DDF0ED05BDF0CD0D8
:1005400004011F5305E128501E5D02E21EC428F07D
:10055000010E1D6E000151DF1EEF04F00601FD5378
:1005600006E1040E246E0001EADE0DD10601050E3F
:10057000246E040E0701006F980E0601FF6F010E36
:10058000FE6FFE510F08D8A0FED0FEC606F7000190
:10059000A5DE0701016B036A0601FE51F2CF05F7E4
:1005A000F29E000192DD070105BFF28EFF0871E0A7
:1005B000040E016FD8900601FE35036AF2CF05F7ED
:1005C000F29E0001AADD0900F5CF03F0070105BF87
:1005D000F28E026F03C003F7496BFEC648F74B6B00
:1005E000080E4A6F000169DE01C005F7010E070120
:1005F0000124016E000E0220036E01C0E9FF040E0B
:100600000324EA6E02C7EFFF496BFEC648F74B6B47
:10061000080E4A6F000151DE01C005F7020E070106
:100620000124016E000E0220036E01C0E9FF040EDA
:100630000324EA6E00C7ECFFED52FFC6EFFFD8902F
:100640000601FE35036AF2CF05F7F29E000165DD73
:100650000900F5CF03F0070105BFF28E0601FF2761
:10066000035007010023880E046F03B1048103B314
:100670000483496BFEC648F74B6B080E4A6F0001B6
:100680001CDE070101C0E9FF040E0224EA6E04C764
:10069000EFFF036A0601FE51F2CF05F7F29E00015B
:1006A00004DD070105BFF28EFF084EE00183496BB0
:1006B000FEC648F74B6B080E4A6F0001FEDD02C014
:1006C00006F701C005F7040E07010527000E0623F3
:1006D000020E0525016E000E0621036E01C0E9FF22
:1006E000040E0324EA6E00C7ECFFED52FFC6EFFFD5
:1006F000D8900601FE35036AF2CF05F7F29E00019D
:10070000F4DC0900F5CF03F0070105BFF28E060106
:10071000FF27035007010023496BFEC648F74B6BC8
:10072000080E4A6F0001C9DD02C006F701C005F7D7
:10073000040E07010527000E062305C7E9FF040E76
:100740000625EA6E400EEF6E0151060802E10E0E1C
:10075000016F036A0601FE51F2CF05F7F29E000118
:10076000A4DC070105BFF28E0108D8A40189036A41
:100770000601FE51700FE96E0F0E0320EA6E01C7ED
:10078000EFFFFE2BFED6000116EF04F00401195115
:1007900000010DE0010A15E0020A20E0060A2AE045
:1007A000030A31E00E0A30E0010A36E045D01FC0EE
:1007B00058F40401596B020E0701006F000117DEA7
:1007C0003DD004011A2D07D0010E1F160701006B42
:1007D00000010DDE02D000010DDE30D004011A2D23
:1007E00006D01F820701006B000101DE02D000016C
:1007F00001DE24D0020E1D6E1AC426F00701006B24
:100800000001F5DD1BD04AD61EC058F4010E0701C9
:10081000006F0001ECDD12D004011A5101080AE357
:100820001AC41EF01AC4FDF6000198D60701006B29
:100830000001DDDD000102D0DDDD00D0F3EF05F0C9
:100840001EC0FDF604011951000105E00A0A0CE082
:10085000010A31E045D00401586B596B020E0701C3
:10086000006F0001C4DD3ED00601FD5321E0010E02
:10087000FD5D036AF2CFFEF6F29E000190DC0601F8
:10088000FEBFF28E016E04011C5DD8A002D00601ED
:100890000FD0036A1C51290FE96E000E0320EA6E87
:1008A000EFCF58F4010E0701006F0001A0DD02D068
:1008B0000001A0DD17D00601FD530FE0036A04011B
:1008C0001C51290FE96E000E0320EA6E1AC4EFFFD7
:1008D0000701006B00018BDD02D000018BDD02D02F
:1008E00089DD00D0F3EF05F00601FE91FDBFFE812A
:1008F000FD9FFEA113D0036AFD51F2CFFFF6F29ED9
:10090000000155EC00F00601FFBFF28EFF0802E186
:10091000000E01D0010E016E13D012D0036AFD51FA
:10092000F2CFFFF6F29E000165EC00F00601FFBF7A
:10093000F28EFF0802E1000E01D0010E016E00D020
:10094000000154EF05F00601FE91FDBFFE81FD9F01
:10095000FEA11DD00701496BFDC648F74B6B080E81
:100960004A6F0001AADC02C000F701C0FFF6040EC6
:100970000601FF27000E07010023FFC6E9FF040E52
:1009800007010025EA6E880EEF6E11D006010701FF
:10099000496BFDC648F74B6B080E4A6F00018DDCB2
:1009A00001C0E9FF040E07010224EA6EEF6A0001AC
:1009B00063EF05F00601FE91FDBFFE81FD9FFEA1E4
:1009C0001DD00701496BFDC648F74B6B080E4A6FF7
:1009D000000173DC02C000F701C0FFF6040E06013F
:1009E000FF27000E07010023FFC6E9FF040E0701E1
:1009F0000025EA6E840EEF6E12D006010701496BE6
:100A0000FDC648F74B6B080E4A6F000156DC01C06B
:100A1000E9FF040E07010224EA6E840EEF6E000166
:100A20006BEF05F00601FE91FDBFFE81FD9FFEA16B
:100A30001BD00701496BFDC648F74B6B080E4A6F88
:100A400000013BDC02C001F701C000F7040E070102
:100A50000027000E012300C7E9FF040E0125EA6EFE
:100A6000EFCFFFF6060112D00701496BFDC648F72C
:100A70004B6B080E4A6F000120DC070101C0E9FF43
:100A8000040E0224EA6EEFCFFFF60601FFAF02D09C
:100A9000FFB502D0000E01D0010E016E000177EF0C
:100AA00005F01CC4FDF620D701522EE004011951B7
:100AB000010A000105E0020A0BE0030A11E022D05E
:100AC0001CC4FDF640D70701006B000190DC1CD070
:100AD0001CC4FDF66FD70701006B000188DC14D041
:100AE0000401586B596B1CC4FDF600019BD70152E1
:100AF00003E0010E0401586F020E0701006F0001B0
:100B000076DC02D077DC00D0F3EF05F0FE0E256E28
:100B1000000C04011C2D01D002D01C534EE11951D0
:100B200000010BE0010A0DE0210A1CE0010A1FE0B0
:100B3000030A30E0010A35E03DD0010E836FE6DFA5
:100B40003BD0040EEA6E580EE96EE26A340EE16E96
:100B5000080E016EE6CFEEFF012EFCD71EC400F793
:100B600046DC2AD0020E836F8081D0DF25D0040EB0
:100B7000EA6E580EE96EE26A2B0EE16E070E016E08
:100B8000E6CFEEFF012EFCD7070E0701006F000134
:100B90002EDC12D01AC481F00701006B000127DCA3
:100BA0000BD01AC433F01BC432F00701006B0001F4
:100BB0001EDC02D01FDC00D004010001F3EF05F0C1
:100BC0001D6A040118517F0B000107E0010A06E0CD
:100BD000030A05E0230A04E004D0D8D531D661D752
:100BE00098D708DC00D061EF08F00701496BFDC61B
:100BF00048F74B6B080E4A6F00015DEC01F00701EE
:100C000001C0E9FF040E0224EA6EEFCFFFF60601F1
:100C1000FE51020806E1FFAD02D0FE6B02D0010ECC
:100C2000FE6FFE5103081EE1840EFF6F0701496B42
:100C3000FDC648F74B6B080E4A6F00015DEC01F0F2
:100C400002C003F701C002F7040E07010227000EDD
:100C5000032302C7E9FF040E0325EA6E840EEF6E3C
:100C600009D00601FE2D03D0C80EFF6F02D0880EFA
:100C7000FF6F0701D8900601FD35036AF2CF02F736
:100C8000F29E00018DEC00F00900F5CF03F00701A2
:100C900002BFF28E006F03C001F7496BFDC648F733
:100CA0004B6B080E4A6F00015DEC01F001C002F7CA
:100CB000010E07010124016E000E0220036E01C027
:100CC000E9FF040E0324EA6E00C7EFFF01A103D081
:100CD0000601FF81070101A303D00601FF8307017D
:100CE000496BFDC648F74B6B080E4A6F00015DEC7F
:100CF00001F0070101C0E9FF040E0224EA6EFFC6FD
:100D0000EFFF0001000C036A07014751700FE96E05
:100D10000F0E0320EA6EEF521BE0496B47C748F7FE
:100D20004B6B080E4A6F00015DEC01F002C049F701
:100D300001C048F7040E07014827000E492348C7A1
:100D4000E9FF040E4925EA6EEFCF48F748AF02D01D
:100D5000000E01D0010E016E0001000C42C747F7E2
:100D6000D2DF0152D8B486D00701496B42C748F799
:100D70004B6B080E4A6F00015DEC01F002C048F7B2
:100D800001C047F7040E07014727000E4823010E54
:100D90004725016E000E4821036E01C0E9FF040ED5
:100DA0000324EA6E43C7EFFF4551020820E1496B77
:100DB00042C748F74B6B080E4A6F00015DEC01F02B
:100DC00002C048F701C047F7040E07014727000E8D
:100DD000482347C7E9FF040E4825EA6EEFCF46F7E0
:100DE00046AD02D0456B02D0010E456F1AD0455179
:100DF000040817E1496B42C748F74B6B080E4A6F6E
:100E000000015DEC01F0070101C0E9FF040E0224BE
:100E1000EA6EEFCF46F746AD03D0010E456F01D025
:100E2000456B452D03D0C80E466F02D0880E466F25
:100E300044B1468144B34683496B42C748F74B6B84
:100E4000080E4A6F00015DEC01F002C048F701C0D6
:100E500047F7040E07014727000E482347C7E9FF5D
:100E6000040E4825EA6E46C7EFFF010E016E05D05D
:100E700000D00001000E016E07010001000C83513B
:100E8000010A03E0030A15E028D0EA6A340EE96E8D
:100E9000040EE26E180EE16E080E016EE6CFEEFF54
:100EA000012EFCD70701006B0001F7EC01F0836B0A
:100EB00018D0EA6A2B0EE96E040EE26E180EE16E8F
:100EC000070E016EE6CFEEFF012EFCD7836B070104
:100ED000006B0001F7EC01F004D0836B42EC01F0F1
:100EE00000D0A6EF07F00701496BFEC648F74B6B31
:100EF000080E4A6F00015DEC01F002C000F701C06E
:100F0000FFF6010E06010124016E000E070102200A
:100F1000036E01C0E9FF040E0324EA6E036AEFCFFB
:100F200001F003C002F000019DEF07F07D817F6BAF
:100F3000020E0601FE6F0001D6D701C07EF0ADEFB4
:100F400007F00601FD5304E1000199D706D0060120
:100F5000FD51020803E10001E9D706010001000C80
:100F6000FEC66EFF0601FE5303E0040E246E02D09F
:100F7000020E246E0001C2EF07F01E6A1D6A26C031
:100F8000FEF6EED73BEF08F03AC747F7BCDE01525A
:100F90004AE00701496B3AC748F74B6B080E4A6FA6
:100FA00000015DEC01F002C043F701C042F7040EFE
:100FB00007014227000E4323020E4225016E000E58
:100FC0004321036E01C0E9FF040E0324EA6EECCF57
:100FD00003F0ED52EFCF40F703C041F741C7EAFFFE
:100FE00040C7E9FF3CC7E2FF3BC7E1FF3EC702F055
:100FF0003DC701F0015202E0022A02D0025206E08F
:10100000E6CFEEFF012EFCD7022EFAD73AC742F701
:101010003EC744F73DC743F73FC745F700019EDE93
:10102000015003D000D0000E016E000C020E07012B
:101030003A6F3C6B3C0E3B6F3E6B7CC03DF7020E43
:101040003F6F0001A1DF7CC082F07C6B000C7C5301
:1010500001E0ECDF42EF08F00601FD530EE11D2C2C
:1010600005D00001FDEC01F006D006011D5002087C
:1010700003E1000182D7060106D0FD51020803E119
:101080000001E5D706010001000C6C300601FB6F82
:10109000FB33FB331F0EFB176C524EE10401005172
:1010A0003C0B0601FC6F430E040100170001D5EC58
:1010B00001F00601FC51340822E10401046B000137
:1010C0007FD56D98253C07D00601FD6B030EFE6FA2
:1010D00000018BDD12D00601FD6B020EFE6F0001D8
:1010E00084DD2550FE0809E00701426B446B25C0F2
:1010F00043F7040E456F000131DE1CD00601FC51A0
:10110000040819E1FD6B00011CDF0601FD6B020EF6
:10111000FE6F00016ADD2550FE080CE0253C01D081
:1011200009D00701426B446B25C043F7010E456FA0
:10113000000114DE06019BD06C5004081DE1430E33
:10114000040104170001D5EC01F0FF0E256E060125
:10115000FD6B000181DF253C01D00AD00701426B05
:10116000446B25C043F7020E456F0001F7DD02D046
:1011700042EC01F07BD006016CB435D00701496B1D
:10118000FBC648F74B6B080E4A6F00015DEC01F09F
:1011900001C0FDF6060101C001F0040E0224036E39
:1011A00001C0FDF6FE6F0701496BFBC648F74B6BAC
:1011B000080E4A6F00015DEC01F001C0E9FF040E6A
:1011C00007010224EA6EEF50430B0601FEC6EAFF58
:1011D000FDC6E9FFEF6E0001D5EC01F0FBC6FDF6A0
:1011E000B0DE44D006010701496BFBC648F74B6BE4
:1011F000080E4A6F00015DEC01F002C0FEF601C06E
:10120000FDF6040E0601FD27000EFE23FDC601F0CB
:10121000040EFE25036EFDC6FDF6FE6F0701496B49
:10122000FBC648F74B6B080E4A6F00015DEC01F0FE
:1012300002C000F701C0FFF6040E0601FF27000EF2
:1012400007010023FFC6E9FF040E07010025EA6E2F
:10125000EF50430B0601FEC6EAFFFDC6E9FFEF6E45
:101260000001D5EC01F0FBC6FDF6F6DE060100013B
:101270006EEF09F0245201E13AD0685238E068A4D8
:1012800004D069A402D03AEF01F06DA201D02FD0B2
:1012900068AA04D069AA02D052EF01F068A204D073
:1012A00069A202D059EF01F068A004D069A002D071
:1012B000DAEF01F068A804D069A802D0EFEF01F0DE
:1012C00068AC04D069AC02D0F4EF01F00601FA6B0F
:1012D00068A606D069A604D00001D7D602D00601C0
:1012E00005D00601FA51FA2B0308F2E20001A19A97
:1012F00032EF00F06D6A696A080E6F6E9450300923
:101300000601946E246A186AF2BE188EF29E0001DD
:10131000BFEC01F018BEF28E8FEF09F0EBD7B5EFFE
:1013200009F0186AF2BE188EF29EBFEC01F018BEEA
:10133000F28E6D6A140E6F6E696A6D86010E246EF0
:10134000A5EF09F06DB601D0ECD7242C0BD06DBA07
:1013500009D0686A696AA08AC00EF212110E696E1D
:10136000020E246EB6EF09F0D9D7ECD7245002084C
:10137000FCE1F2EF0FF00601DD91F2BEDD81F29E9D
:1013800000017C513F0802E23F0E7C6F7C517C2BB8
:10139000036A3C0FE96E000E0320EA6EDCC6EFFF25
:1013A000F29E0601DDB1F28E186AF2BE188EF29E30
:1013B000020E0701476F0001A6DC18BEF28E015233
:1013C00007E0186AF2BE188EF29E30DE18BEF28E6A
:1013D00005EF0AF07C513F0815E2186AF2BE188E3C
:1013E000F29E020E0701476F00018DDC18BEF28EDF
:1013F000015207E0186AF2BE188EF29E17DE18BE80
:10140000F28EE8D7DBC6DCF6B6D7000C8E0E006E87
:10141000D9C601F0D8C602F0036A015209E102C040
:1014200001F0026A080E005E015202E1006A08D073
:10143000D89001BE04D0023601360006F9D7019ECD
:10144000000C800ED8A202D00601EF1B0601F46B3F
:10145000F56BEBC6F3F6EF51F31BEA51D8B4DFD0CE
:10146000F26F006EEE51D8B4E3D0F25FD8B483D0FF
:101470003EE3EFC6F8F6F88FF0C6F7F6F1C6F6F6DB
:10148000F56BD890F833F733F633F533F22FF8D7FE
:10149000F3AF03D0F481E0D0F491F291F489060E19
:1014A000EA6EED0EE96EEBD0F499F3BF0AD0F2A12B
:1014B00013D0F833F733F633F533002AD8B4C7D056
:1014C0000BD0F8BF0CD0D890F537F637F737F83790
:1014D0000006D8B4BCD0F5D7F48D6DD0F49DEBC622
:1014E000F3F6EBAF02D0F88FABD0F89FA9D0EEC6E1
:1014F000F2F6EEC600F0EA51F25FEBC6F8F6F88FAE
:10150000ECC6F7F6EDC6F6F6F56BD890F833F73380
:10151000F633F533F22FF8D7F3AF03D0F4839CD032
:10152000F493F291F48B060EEA6EF10EE96EA7D0F9
:10153000F49BF3BF0AD0F2A113D0F833F733F6339C
:10154000F533002AD8B483D00BD0F8BF0CD0D89094
:10155000F537F637F737F8370006D8B478D0F5D72F
:10156000F48F29D0F49FEFC6F3F6EFAF02D0F88FD7
:1015700067D0F89F65D0EFC6F8F6F88FF0C6F7F69B
:10158000F1C6F6F6F3AF04D0F89FF48565D0F49574
:10159000F56BF291060EEA6EED0EE96E70D0F3BFB8
:1015A0001CD0EBC6F3F6F2A106D0F833F733F633CE
:1015B000F533002A4CE0F5AF0BD0F62B09E1F72B01
:1015C00007E1F82B05E1F833F733F633002A3FE063
:1015D000F4BD84D7F4BFC6D71CD0800EF81BF8AF7B
:1015E00004D03AD0EFC6F3F60AD0EBC6F3F6F853C0
:1015F00006E1F75304E1F65302E1006A21D0F8BF97
:1016000008D0D890F537F637F737F837002EF7D7E8
:101610001ED0F3AF02D0F88F13D0F89F11D0EEC6D2
:1016200000F0EFC6F8F6F0C6F7F6F1C6F6F608D009
:10163000EAC600F0EBC6F8F6ECC6F7F6EDC6F6F62D
:10164000F8C601F0F7C602F0F6C603F034D0006A1F
:10165000016A026A036A2FD0F56BF61FF71FF81FA5
:10166000F51FF52B05E1F62B03E1F72B01E1F82B34
:10167000F4B112D7F4B354D7F4B589D7B3D7EF5038
:10168000F62705E3F72B03E1F82BD8B4F281ED52EE
:10169000EF50F72703E3F82BD8B4F281ED52EF5067
:1016A000EFBE01D0800AF827D8B0F281F4B9FCD699
:1016B000F4BB3ED774D70001000C0601EA51D8B440
:1016C000A5D0F66FEE51D8B4A1D0F65F05E37F0E3A
:1016D000F627D8B09BD006D0810EF65FD8A096D062
:1016E000D8B494D0F6C600F0016A026A036AF56BBA
:1016F000EBC6F4F6F48FECC6F3F6EDC6F2F6190E6F
:10170000F66FF151F25F0DE2010EF35F0AE2F45F52
:1017100008E2F55F06E2F52BF42BF32BF151F227EB
:1017200028D0F051F35F12E2010EF45F0FE2F55F93
:101730000DE2F52BF42BF051F327F151F22719E3C9
:10174000F32B17E1F42B15E1F52B13D0EF518009A2
:10175000F45F0EE2010EF55F0BE2F52BEF5180090D
:10176000F427F051F327E9E3F42BE7E1F52BE5D774
:101770000380F62F01D00BD0D890F237F337F4372F
:10178000F537D890033602360136F737BAD7F7A1C6
:1017900006D0D890013202320332F73302D000066D
:1017A00035E0F7BF1ED0D890F237F337F437F5376E
:1017B000F151F25F07E2010EF35F04E2F45F02E22F
:1017C000F55F1AE3F051F35F05E2010EF45F02E208
:1017D000F55F12E3EF518009F45F03E2010EF55F5C
:1017E0000BE3032A09E1022A07E1012A05E1002AA5
:1017F0000DE0013202320332EBC6F6F6EF51F61B72
:10180000F6AF02D0018E06D0019E04D0006A016AB4
:10181000026A036A0001000CB60E006E036A026AD7
:10182000016A0601C251C311C411C51102E1006A67
:101830000DD0D89001BE09D0C237C337C437C537E1
:10184000033602360136002EF4D7019E0001E9EF7F
:1018500011F00601E451D8B471D0006EE851D8B44B
:101860006DD0002604E3810E002668E204D07F0ECE
:10187000005E64E363E0E5C6ECF6E951EC1BE58F3E
:10188000E98FE751EB03F4CFEEF6E651EA03F4CF2C
:1018900003F0F3CFEDF6EB03F350EE27F450ED2316
:1018A000000E0322E751EA03F350EE27F450ED2334
:1018B000000E026A03220222E551EB03F350ED27EA
:1018C000F4500322000E0222E551EA03F3500326EE
:1018D000F4500222000E016A0122E751E903F3509D
:1018E000ED27F4500322000E02220122E651E90303
:1018F000F3500326F4500222000E0122E551E903C1
:10190000F3500226F4500122002A01BE05D0ED3723
:101910000336023601360006000EEDAF0AD0032A68
:1019200002220122015005E1025003E1035001E1CE
:10193000002AECBF018EECAF019E04D0006A016A60
:10194000026A036A0001000CEBC6F2F60601EF51D1
:10195000F21BF2AF05D0D894D890EBBFD8802FD02F
:10196000EBC6F2F6EEC6F3F6EA51F35F06E0F2AF2D
:1019700026D0D850010AD86E22D0EFC6F3F6EB512C
:10198000F35F06E0F2AF1BD0D850010AD86E17D033
:10199000F0C6F3F6EC51F35F06E0F2AF10D0D8508A
:1019A000010AD86E0CD0F1C6F3F6ED51F35F06E0F4
:1019B000F2AF05D0D850010AD86E01D0D8900001FE
:1019C000000CDFC6EDF6DEC6ECF6DDC6EBF6DCC6D7
:1019D000EAF60601F16BF06BEF6BEE6B0001B4DF22
:1019E00001E205E1006A016A026A036A78D0DFC693
:1019F000E3F6DEC6E2F6DDC6E1F6DCC6E0F6060E8C
:101A00000601E96FE00EE86FE8C6E9FFE9C6EAFF04
:101A1000EF50ED6BEC6F7F0EEC27000EED23D890AE
:101A2000ED31EC31E9C6EAFFE8C6E9FFEF6EE3C647
:101A3000E7F6E2C6E6F6E1C6E5F6E0C6E4F6DFC69E
:101A4000EDF6DEC6ECF6DDC6EBF6DCC6EAF6E3C67E
:101A5000F1F6E2C6F0F6E1C6EFF6E0C6EEF60001FA
:101A60002CDED892E3C6EDF6E2C6ECF6E1C6EBF664
:101A7000E0C6EAF603C0F1F602C0F0F601C0EFF6E8
:101A800000C0EEF6DEDC03C0E3F602C0E2F601C001
:101A9000E1F600C0E0F60601E8C6E9FFE9C6EAFFA4
:101AA000EF06E7C6EDF6E6C6ECF6E5C6EBF6E4C6ED
:101AB000EAF6E3C6F1F6E2C6F0F6E1C6EFF6E0C6F6
:101AC000EEF6000141DFD8B402D00601B0D7E4C67B
:101AD00000F0E5C601F0E6C602F0E7C603F065EFE8
:101AE0000EF00601D46BD56BD66BD76BD36BD26B74
:101AF000D351D15DD8A0A8D004E1D051D25DD8B0E7
:101B0000A3D0D235026ED335036E02360336FC0EF7
:101B100002160250CE25E96ECF510320EA6EEFCFB8
:101B2000D8F6ECCFD9F6ECCFDAF6ECCFDBF6EACF8D
:101B3000DDF6E9CFDCF6D882DBC6EDF6DAC6ECF6E8
:101B4000D9C6EBF6D8C6EAF6CDC6F1F6CCC6F0F6A5
:101B5000CBC6EFF6CAC6EEF6000173DCDDC6EAFFBF
:101B6000DCC6E9FF00C0D8F601C0D9F602C0DAF63B
:101B700003C0DBF60601D235026ED335036E0236A2
:101B80000336FC0E02160250CE25E96ECF5103201B
:101B9000EA6EEFCFDEF6ECCFDFF6ECCFE0F6ECCF7F
:101BA000E1F6EACFE3F6E9CFE2F6D882E1C6EDF658
:101BB000E0C6ECF6DFC6EBF6DEC6EAF6CDC6F1F619
:101BC000CCC6F0F6CBC6EFF6CAC6EEF6000139DC9D
:101BD000E3C6EAFFE2C6E9FFDBC6E7F6DAC6E6F6E9
:101BE000D9C6E5F6D8C6E4F603C0EBF602C0EAF6BD
:101BF00001C0E9F600C0E8F62CDEEACFD9F6E9CF5D
:101C0000D8F6D892D7C6EDF6D6C6ECF6D5C6EBF622
:101C1000D4C6EAF603C0F1F602C0F0F601C0EFF652
:101C200000C0EEF60EDCD9C6EAFFD8C6E9FF03C055
:101C3000D7F602C0D6F601C0D5F600C0D4F606012C
:101C4000D22BD8B4D32B54D7D1C6D9F6D0C6D8F618
:101C5000000106EC0AF00601ED6BEC6BEB6B7F0EFE
:101C6000EA6F03C0F1F602C0F0F601C0EFF600C063
:101C7000EEF6000122DD00C0D8F601C0D9F602C0A0
:101C8000DAF603C0DBF603C0E7F602C0E6F601C0F1
:101C9000E5F600C0E4F6D7C6EBF6D6C6EAF6D5C63A
:101CA000E9F6D4C6E8F6D5DD00C0D8F601C0D9F60D
:101CB00002C0DAF603C0DBF603C0DFF602C0DEF6D0
:101CC00001C0DDF600C0DCF67CD603C0D7F602C04A
:101CD000D6F601C0D5F600C0D4F6D4C600F0D5C6FD
:101CE00001F0D6C602F0D7C603F0000C0601DB51A6
:101CF000B608DB6F036ADCC6DFF6DC8FD890DC3316
:101D0000DD33DE330332023201320032DB2FF6D70D
:101D1000DFAF0BD0001E011E021E031E002AD8B426
:101D2000012AD8B4022AD8B4032A000103EF0FF025
:101D3000006A016A026A036A0601E36BE46BE56B01
:101D4000E66BE251E111E011DF112CE0200EE76FAC
:101D5000D890DB37DC37DD37DE37E337E437E5377C
:101D6000E637E251E65D08E1E151E55D05E1E0516C
:101D7000E45D02E1DF51E35D0FE3DF51E35FE0513A
:101D8000D8A0E03DE45FE151D8A0E13DE55FE2513C
:101D9000D8A0E23DE65FD880003601360236033631
:101DA000E72FD6D7060EEA6EE30EE96E0001000CAF
:101DB000E9500601D36FD251D56F1BE0D1C6E7F6CB
:101DC000D0C6E6F6CFC6E5F6CEC6E4F6EB6BEA6B18
:101DD000200EE96F820EE86F00013BDD03C0D1F6F3
:101DE00002C0D0F601C0CFF600C0CEF60601D52F56
:101DF000E5D7D1C6DEF6D0C6DDF6CFC6DCF6CEC658
:101E0000DBF6000173D703C0D1F602C0D0F601C0E3
:101E1000CFF600C0CEF60601D1AF0DD0D307D38BDD
:101E2000CE1FCF1FD01FD11FCE2BD8B4CF2BD8B4ED
:101E3000D02BD8B4D12B3B0EDA6F9A0ED96FCA0EC5
:101E4000D86FD76B0A0ED56FD251D8B4D32BD1C669
:101E5000DEF6D0C6DDF6CFC6DCF6CEC6DBF6DAC6D9
:101E6000E2F6D9C6E1F6D8C6E0F6D7C6DFF600013D
:101E70005FDF0150EFCFCEF6ECCFCFF6ECCFD0F650
:101E8000ECCFD1F6005213E10601D229D55DD8A4DA
:101E900002D000010CD0D3510DE00F0BD55D01E055
:101EA00044E2D3BF42D0D3BD05D0200E37D0200EA0
:101EB0000601D317D3AB0FD0D39BD251D8A4D307ED
:101EC0000050D36F2D0EDB6F0001EAEC09F0060124
:101ED000D351006ED36BD251D55D0DE10050D36F5D
:101EE0002E0EDB6F0001EAEC09F00601D351006E03
:101EF000200ED317000E300ED3AB10D0D39BD2518F
:101F0000D8A4D3070050D36F2D0EDB6F0001EAEC8D
:101F100009F00601D351006ED36B300E002600C0CD
:101F2000DBF60001EAEC09F00601DAC6DEF6D9C6F6
:101F3000DDF6D8C6DCF6D7C6DBF6E26BE16BE06B0C
:101F40000A0EDF6F0001F4DE03C0DAF602C0D9F634
:101F500001C0D8F600C0D7F60601D52F78D700010A
:101F6000000CF86AD09E088EEA6AE96AC150C00B7C
:101F70000F09C16E070EB46E216A040E226E0C0E9C
:101F8000236E246A286A7C6B836BF18EB098C69AA4
:101F9000949E93809392010EC66E000EC76ED190F0
:101FA000870ED56ECD6A000ECA6E000ECB6EB16A7A
:101FB000070EB46E9250926E130E006E002EFED776
:101FC00000D0B450A19CB56AF28AC00EF212C15082
:101FD000C00B1C09C16EC090C082C084C08EC2807C
:101FE000B4EF09F080A1FED71C6A1B6A1A6A196A4D
:101FF000D76AD66A0301B16BB15100010FEC01F051
:102000000301B12B006EE8CFDBF60001EAEC09F02A
:10201000250E0301B15DF0E1000180A1E0D20301D2
:10202000B06BB0516308D8A06BD1000E016EC250E6
:10203000C30B0110C26E130E006E002EFED700D02F
:10204000186AF2BE188EF29E0701496BB0C348F7BA
:102050004B6B040E4A6F00015DEC01F018BEF28E6E
:1020600002C003F00150840FE96E000E0220EA6EF8
:10207000C282C2B2FED7C4CFD9F6C3CFD8F6000110
:1020800006EC0AF000C0EFFF01C0ECFF02C0ECFF5D
:1020900003C0ECFF186AF2BE188EF29E0701496B6E
:1020A000B0C348F74B6B040E4A6F00015DEC01F0C2
:1020B00018BEF28E02C003F00150840FE96E000ECC
:1020C0000220EA6EEFCF00F0ECCF01F0ECCF02F08F
:1020D000ECCF03F0EACFB2F3E9CFB1F3D892A7C3C4
:1020E000EDF6A6C3ECF6A5C3EBF6A4C3EAF603C06F
:1020F000F1F602C0F0F601C0EFF600C0EEF621ECFA
:102100000AF0B2C3EAFFB1C3E9FF03C0A7F302C0FC
:10211000A6F301C0A5F300C0A4F3040E016EC250E3
:10212000C30B0110C26E130E006E002EFED700D03E
:10213000186AF2BE188EF29E0701496BB0C348F7C9
:102140004B6B040E4A6F00015DEC01F018BEF28E7D
:1021500002C003F00150140FE96E020E0220EA6E75
:10216000C282C2B2FED7C4CFD9F6C3CFD8F600011F
:1021700006EC0AF000C0EFFF01C0ECFF02C0ECFF6C
:1021800003C0ECFF186AF2BE188EF29E0701496B7D
:10219000B0C348F74B6B040E4A6F00015DEC01F0D1
:1021A00018BEF28E02C003F00150140FE96E020E49
:1021B0000220EA6EEFCF00F0ECCF01F0ECCF02F09E
:1021C000ECCF03F0EACFB2F3E9CFB1F3D892ABC3CF
:1021D000EDF6AAC3ECF6A9C3EBF6A8C3EAF603C072
:1021E000F1F602C0F0F601C0EFF600C0EEF621EC09
:1021F0000AF0B2C3EAFFB1C3E9FF03C0ABF302C008
:10220000AAF301C0A9F300C0A8F3080E016EC250E2
:10221000C30B0110C26E130E006E002EFED700D04D
:10222000186AF2BE188EF29E0701496BB0C348F7D8
:102230004B6B040E4A6F00015DEC01F018BEF28E8C
:1022400002C003F00150200FE96E050E0220EA6E75
:10225000C282C2B2FED7C4CFD9F6C3CFD8F600012E
:1022600006EC0AF000C0EFFF01C0ECFF02C0ECFF7B
:1022700003C0ECFF186AF2BE188EF29E0701496B8C
:10228000B0C348F74B6B040E4A6F00015DEC01F0E0
:1022900018BEF28E02C003F00150200FE96E050E49
:1022A0000220EA6EEFCF00F0ECCF01F0ECCF02F0AD
:1022B000ECCF03F0EACFB2F3E9CFB1F3D892AFC3DA
:1022C000EDF6AEC3ECF6ADC3EBF6ACC3EAF603C075
:1022D000F1F602C0F0F601C0EFF600C0EEF621EC18
:1022E0000AF0B2C3EAFFB1C3E9FF03C0AFF302C013
:1022F000AEF301C0ADF300C0ACF30301B02B91D637
:10230000A7C3EDF6A6C3ECF6A5C3EBF6A4C3EAF6A5
:102310000601F16BF06B480EEF6F850EEE6F00015A
:102320005DEC0BF003C0A7F302C0A6F301C0A5F358
:1023300000C0A4F3ABC3EDF6AAC3ECF6A9C3EBF659
:10234000A8C3EAF60601F16BF06B480EEF6F850E3D
:10235000EE6F00015DEC0BF003C0ABF302C0AAF31B
:1023600001C0A9F300C0A8F3AFC3EDF6AEC3ECF60D
:10237000ADC3EBF6ACC3EAF60601F16BF06B480EA9
:10238000EF6F850EEE6F00015DEC0BF003C0AFF355
:1023900002C0AEF301C0ADF300C0ACF31AC0B5F398
:1023A00019C0B4F30301B26BB36BD650D7CF03F0AF
:1023B000B227D750B323000EB423B523B5C3C5F657
:1023C000B4C3C4F6B3C3C3F6B2C3C2F600010CEF84
:1023D0000CF003C0EDF602C0ECF601C0EBF600C055
:1023E000EAF60601F16B240EF06F740EEF6F8C0E9F
:1023F000EE6F00015DEC0BF000C0B2F301C0B3F36F
:1024000002C0B4F303C0B5F3A7C3CDF6A6C3CCF6A0
:10241000A5C3CBF6A4C3CAF60601CF6B840ECE6F5C
:10242000D16B640ED06F000171EC0DF000C0B6F3FB
:1024300001C0B7F302C0B8F303C0B9F3ABC3CDF624
:10244000AAC3CCF6A9C3CBF6A8C3CAF6020E0601EE
:10245000CF6F140ECE6FD16B640ED06F000171EC94
:102460000DF000C0BAF301C0BBF302C0BCF303C05F
:10247000BDF3AFC3CDF6AEC3CCF6ADC3CBF6ACC3A4
:10248000CAF6050E0601CF6F200ECE6FD16B640E1B
:10249000D06F000171EC0DF000C0BEF301C0BFF3BE
:1024A00002C0C0F303C0C1F3060EE96EB5C3D1F696
:1024B000B4C3D0F6B3C3CFF6B2C3CEF6030E060153
:1024C000D26F000175DC200E0601DB6F0001EAEC23
:1024D00009F0030EE96EA7C3D1F6A6C3D0F6A5C3D3
:1024E000CFF6A4C3CEF60601D26F000161DC200E48
:1024F0000601DB6F0001EAEC09F0030EE96EB9C3D7
:10250000D1F6B8C3D0F6B7C3CFF6B6C3CEF6060140
:10251000D26F00014DDC200E0601DB6F0001EAECFA
:1025200009F0030EE96EABC3D1F6AAC3D0F6A9C376
:10253000CFF6A8C3CEF60601D26F000139DC200E1B
:102540000601DB6F0001EAEC09F0030EE96EBDC382
:10255000D1F6BCC3D0F6BBC3CFF6BAC3CEF60601E4
:10256000D26F000125DC200E0601DB6F0001EAECD2
:1025700009F0030EE96EAFC3D1F6AEC3D0F6ADC31A
:10258000CFF6ACC3CEF60601D26F000111DC200EEF
:102590000601DB6F0001EAEC09F0030EE96EC1C32E
:1025A000D1F6C0C3D0F6BFC3CFF6BEC3CEF6060188
:1025B000D26F0001D8EC0EF0200E0601DB6F000197
:1025C000EAEC09F00A0E0601DB6F0001EAEC09F003
:1025D0000D0E0601DB6F0001EAEC09F01ED502D5F5
:0225E0000300F6
:020000040030CA
:0E0000003CCE390E0087A1000FC00FE00F406C
:00000001FF
